:0A00000075817F7401F58F02002E58
:10002B0002409DC294D294C2A4D2A57532007533FE
:10003B000075340075350075360075370075630033
:10004B00756400754500754601754701756001754E
:10005B006101756201754800754900754A00754B61
:10006B0000754C01C233754D00755A0075590075FA
:10007B005C00755B007553007554007552F0754E3E
:10008B0000754F00755000755D00C20AC22EC20C80
:10009B00C210C211C214C215C212C213C20FC216B1
:1000AB00C217C218C219C21AC21BC21CC21DC21E61
:1000BB00C21FC220D209C234C235D236740090009E
:1000CB0030F0900031F0900032F0900033F090005F
:1000DB0034F07400900035F0900036F090027F748D
:1000EB0000F0A37404F0A37407F0A37409F090015B
:1000FB00207416F09001217401F012384E12385A08
:10010B009001177401F09001227401F09001237497
:10011B0001F09001277401F09001187401F0900127
:10012B00247401F09001197401F090011A7401F01C
:10013B0090011B7401F090011F7401F090011C746D
:10014B0001F090011D7401F090011E7401F09001FB
:10015B00297401F0753C00753D0012094F7538008C
:10016B001204D912037A1204E67538001201FD123B
:10017B00407712074BC2A1120ABB120AC5120ACF53
:10018B00120AED120B7B120B991204BF1204D91237
:10019B0001FD1201FD753C30753D08123DE1753CCA
:1001AB0000753D00123D7C124037121D8C121E470C
:1001BB00122426C202C203123266122063123816B0
:1001CB001231F61234AD1220C2900122E0B40306B4
:1001DB001233150201E650F81224BF121C64121FD1
:1001EB00C21224070201CB783279FF0000D9FCD868
:1001FB00F822786479FF0000D9FCD8F82278967938
:10020B0096D9FED8FA2278FF799BD9FED8FA2278B4
:10021B000A790AD9FED8FA22E627F5270809E63724
:10022B00F528782722C3E697F5270809E697F528DE
:10023B007827228627872908098628872A1202C34E
:10024B00782C22862C08862D08862E08862F872947
:10025B0009872A1202667827792E227530007531AC
:10026B00101202A812027912029CD531F422C3E5B6
:10027B002E9529E52F952AE5309400500122E52E85
:10028B009529F52EE52F952AF52FE5309400F530BD
:10029B0022B3E52733F527E52833F52822C3E52CD0
:1002AB0033F52CE52D33F52DE52E33F52EE52F33D8
:1002BB00F52FE53033F53022E5278529F0A4F52C11
:1002CB0085F02DE528852AF0A4F52E85F02FE5285D
:0A02DB008529F0A4252DF52DE52E50
:1002E50035F0F52EE52F3400F52FE527852AF0A406
:1002F500252DF52DE52E35F0F52EE52F3400F52FBE
:1003050022E538B4101120010ED201C28174C01249
:10031500034AD282C28222E538B4200FC28174809A
:1003250012034AD282C28275380022C201A200920B
:1003350081900000E5822538F582E012034AD282D9
:10034500C282053822F954F053800F4280D282C20E
:1003550082E9C454F053800F4280221201FD22121B
:1003650001FD1201FD1201FD1201FD1201FD120137
:10037500FD1201FD22C282120360120360C281C216
:10038500831201FDD282C287C286D285D284120130
:10039500FDC282120360C281C2831201FDD282C2F4
:1003A50087C286D285D2841201FDC282120360C241
:1003B50081C2831201FDD282C287C286D285D284D0
:1003C5001201FDC282120360C281C2831201FDD2F5
:1003D50082C287C286D285C2841201FDC2821203FF
:1003E50060C281C2831201FDD282C287C286D285D4
:1003F500C2841201FDC282120360C281C28312014E
:10040500FDD282D287C286C285C2841201FDC28214
:10041500120360C281C2831201FDD282C287C286E5
:10042500C285C2841201FDC282120360C281C283E9
:100435001201FDD282D287D286D285C2841201FDF5
:10044500C282120360C281C2831201FDD282C287B9
:10045500C286C285C2841201FDC282120360C281B6
:10046500C2831201FDD282C287C286C285D284129E
:1004750001FDC282120360C281C2831201FDD282D4
:10048500C287C286C285C2841201FDC28212036080
:10049500C281C2831201FDD282C287D286D285C2B1
:1004A500841201FDC282120360D2002205A2E493E8
:1004B500A305A2F0A3DBF505A222900F5005A2909B
:1004C50000007B200204B1900F7005A29000007B14
:1004D500200204B1900FC005A29000007B20020409
:1004E500B1C283C281744012034AD282C28212020F
:1004F50011D281740012034AD282C282120211D231
:1005050081741E12034AD282C282120211D28174F0
:100515001E12034AD282C282120211D281741E12A5
:10052500034AD282C282120211D281741E12034A78
:10053500D282C282120211D281741E12034AD28261
:10054500C282120211D281741E12034AD282C28261
:10055500120211C283C281744812034AD282C28236
:10056500120211D281740412034AD282C28212028B
:1005750011D281740E12034AD282C282120211D2A2
:1005850081741512034AD282C282120211D2817479
:100595000412034AD282C282120211D28174041259
:1005A500034AD282C282120211D281740412034A12
:1005B500D282C282120211D281740412034AD282FB
:1005C500C282120211D281740012034AD282C282FF
:1005D500120211C283C281745012034AD282C282AE
:1005E500120211D281740412034AD282C28212020B
:1005F50011D281740412034AD282C282120211D22C
:1006050081740412034AD282C282120211D2817409
:100615000412034AD282C282120211D281741512C7
:10062500034AD282C282120211D281740E12034A87
:10063500D282C282120211D281740412034AD2827A
:10064500C282120211D281740012034AD282C2827E
:0E065500120211C283C281745812034AD2826B
:10066300C282120211D281740412034AD282C2825C
:10067300120211D281740E12034AD282C282120272
:1006830011D281741512034AD282C282120211D28C
:1006930081740412034AD282C282120211D281747B
:1006A3001512034AD282C282120211D281740E122F
:1006B300034AD282C282120211D281740412034A03
:1006C300D282C282120211D281740012034AD282F0
:1006D300C282120211222430F02275F00A84AFF094
:1006E30075F00A84E5F02430F0EF2430A3F022758E
:1006F300F00A84AFF075F00A842430F0E5F024307A
:10070300A3F0EF2430A3F0221206F2A3742CF0EE30
:100713002430A3F022D281C2831201FDD282D28778
:10072300D286D285D2841201FDC282120360D281A5
:10073300C2831201FDD282D287D286D285D284129D
:1007430001FDC282120360221204D91201FD1201BB
:10075300FD1201FD1201FD1201FD1201FD1201FD49
:100763001204BF753C24753D001201FD1201FD7595
:100773003C30753D001201FD1201FD753C20753DB5
:10078300021201FD1201FD753C20753D081201FDA9
:100793001201FD753C20753D201201FD1201FD750E
:1007A3003C20753D801201FD1201FD753C20753D15
:1007B300101201FD1201FD753C20753D041201FD6F
:1007C3001201FD753CA0753D001201FD1201FD757E
:1007D3003C60753D001201FD1201FD753C28753D1D
:1007E300001201FD1201FD753C22753D001201FD51
:1007F3001201FD753C20753D001201FD1201FD75CE
:100803003C20753D001201FD1201FD753C20753D34
:10081300401201FD1201FD753C21753D001201FDE1
:100823001201FD753C20753D011201FD1201FD759C
:100833003C20753D001204CC1201FD1201FD120192
:10084300FD1201FD1201FD1201FD1201FD1201FD58
:100853001201FD1201FD1201FD1201FD1201FD1233
:1008630001FD1201FD1201FD1201FD1201FD120134
:10087300FD1201FD1204D91201FD1201FD1201FD49
:100883001201FD221201FD1201FD1201FD1201FDF3
:100893001201FD1201FD1201FD1201FD1201FD12F3
:1008A30001FD1201FD1201FD1201FD1201FD1201F4
:1008B300FD1201FD1201FD1201FD1201FD1201FDE8
:1008C3001201FD1201FD1201FD1201FD1201FD12C3
:1008D30001FD1201FD1201FD1201FD1201FD1201C4
:1008E300FD1201FD1201FD1201FD1201FD1201FDB8
:1008F3001201FD1201FD1201FD1201FD2220B204BD
:100903007539002220B103D2042275390122E53959
:10091300B53A0485393A22B4001920040A053B8507
:10092300393AD206D20222153BC20485393AD2069D
:10093300D2032220040A153B85393AD206D2032278
:10094300053BC20485393AD206D20222C2B3C2B4ED
:10095300C2B5E53CF4200E0244FE7F083392B6D2C2
:10096300B5C2B5DFF7B2B30000C2B3E53DF4200E64
:100973000244FE79083392B6C2B5D2B5D9F7D2B4E0
:100983000000C2B422C293D2937908C290A29133D9
:10099300D290D9F7F53EC293D2937908C290A2922E
:1009A30033D290D9F7F53F22E582C4540FF9E5839A
:1009B300C46922E5820303543FF9E583030354C06A
:1009C30069227A0CC2A6D2A3A2C133C933C9C2A376
:0E09D300DAF2F8D2A622C2A3C2A63392A7D2AD
:1009E100A3DAF5C2A31209C5E95403F9227A057401
:1009F100C01209D9F5838882227A0574C81209D9EF
:100A0100F5838882227A0574D01209D9F583888208
:100A1100227A0574D81209D9F58388822285823217
:100A210085833375340075350078327536787537BE
:100A310000793612023E8552367537037936120235
:100A41004EE6228582328583337534007535007810
:100A510032753604753700793612022386320886DC
:100A61003375340075350078327536E8753703799A
:100A71003612023E753655753721793612024EE629
:100A8100228582328583337534007535007832755D
:100A91003611753700793612024EE62222C2A0E8DD
:100AA100120AAFE9120AAFEA120AAFD2A0227B08FA
:100AB100D2A13392A2C2A1DBF7227840790F7A004A
:100AC100120A9E227869790F7A00120A9E2278779B
:100AD10079007A00120A9E22782F79FF7AF0120AA1
:100AE1009E22782F79807A00120A9E22782F79002F
:100AF1007A00120A9E22782FF97A00120A9E227831
:100B01002F791F7A80120A9E22782F793F7A00125C
:100B11000A9E22782F79FC7A00120A9E22E583C46C
:100B210054F0F9E582C4FA540F49F9EA54F0FA2273
:100B3100120B1E7800120A9E22120B1E7801120A55
:100B41009E22120B1E7802120A9E22120B1E78039D
:100B5100120A9E22120B1E78A0120B5E22C296E888
:100B6100120B6FE9120B6FEA120B6FD296227B0800
:100B7100D2A1339295C2A1DBF722782779007A00BE
:100B8100120B5E2278A079FF7AF0120B5E2278A018
:100B910079807A00120B5E2278A079007A00120B1C
:100BA1005E2278A0791F7A80120B5E2278A0793FAD
:100BB1007A00120B5E2278A079FC7A00120B5E2279
:100BC100F532753300783275362275370079361271
:100BD100023E868208868322F532753300783275AB
:100BE1003622753700793612023E868208868322C4
:100BF100120E82F532753300783275362A75370058
:100C0100793612023E868208868322F532753300D8
:100C11007832753620753700793612023E868208A1
:100C2100868322900030E004B410027400F090003A
:100C310020A98229F582E022900034E0FA90003167
:100C4100E004B40F0274FFF0900F30932A90003447
:100C5100F0900033E004B410027400F0F990003415
:100C6100E0FA900020E58229F582EAF02290003432
:100C7100E0FA900032E004B4110274FFF0900F3FEB
:100C8100932A900034F0120C5222120C2454016069
:100C910008120C24541F246022747F22F974FF89E6
:100CA100F084F5F0120C248422120C2475F02084B7
:100CB10022120C2475F03384240122120C2475F0C5
:100CC1002084240122120C2475F03F842401221275
:100CD1000C2475F03384240322120C2475F0108443
:100CE10022120C2475F01F8422120C2475F020842A
:100CF100F8120C2475F03F842822120C245401753B
:100D0100F00CA422120C2475F0558475F00CA42269
:100D1100B40101225003740122B4070122500122BF
:100D2100740722B40101225003740122B40A012282
:100D3100500122740A22B40101225003740122B429
:100D41000D0122500122740D22B4010122500374BD
:0E0D51000122B4100122500122741022B401BC
:100D5F0001225003740422B40401225001227401B1
:100D6F0022B40101225003740A22B40A0122500155
:100D7F0022740122B40101225003741822B4180105
:100D8F0022500122740122B4010122500374012266
:100D9F00B43A0122500122743A22B40101225003C5
:100DAF00740122B4460122500122744622B401017B
:100DBF00225003740122B404012250012274042230
:100DCF00B40101225003740122B405012250012203
:100DDF00740522B40101225003740122B4200122B0
:100DEF00500122742022B40101225003740122B455
:100DFF00020122500122740222B401012250037415
:100E0F000122B4020122500122740222B4010122F4
:100E1F005003740122B4050122500122740522B43B
:100E2F000001225003740022B405012250012274E4
:100E3F000522B40001225003740022B40301225092
:100E4F000122740322B4FF03740C22B40B0122504D
:100E5F000122740C22B4FF02EC22B43C0122500197
:100E6F0022EC22B4FF03740022B4030122500122AA
:100E7F00740322B46001224002746022B4FF037431
:100E8F000022B4240122500122742422B401012231
:100E9F005003740122B4180122500122741822B495
:100EAF000101225003740122B40201225001227465
:100EBF000222B40101225003740122B40201225014
:100ECF000122740222F990027AE0F55EE9B4010181
:100EDF00225003740122B55E0122500122E55E22E9
:100EEF00F990027AE0F55EE9B40101225003740132
:100EFF0022B55E0122500122740122B40101225059
:100F0F0003740422B4040122500122740122B4019B
:100F1F0001225003740122B40C0122500122740CDF
:100F2F0022037F2C0C0105712133E6FF0B57681844
:100F3F00BD09A60D004B5D263585B196114093C8AE
:100F4F00D3204620204C20204120204D202045201A
:100F5F002043484F5244204D414348494E4520328B
:100F6F0020202056455253494F4E20312E303120EC
:100F7F00202020286329323031362D32303137206E
:100F8F0020496E697420616C6C2044617461203F4C
:100F9F00204F4B20202020202020202020204E4F8B
:100FAF002020506C65617365207761697420212062
:100FBF002020202020202020202020202020202022
:100FCF002020202020202020202020202020202012
:100FDF00204D4F44452050524F4752414D4D2020F8
:100FEF00204D4F44453C3E202343302020524F4F4D
:100FFF005420205030312020234331202020202026
:10100F00202020503031204449523A646F776E20AF
:10101F004449563A6E6F2020234331200173636198
:10102F006C653A50303120202343312002736361C5
:10103F006C653A50303120202343312003736361B4
:10104F006C653A50303120202043484F52442020C5
:10105F004152502F514152504547494F2020515531
:10106F00414E54204C454E4748542053454C454320
:10107F00544C6973743A41303120202043484F5209
:10108F00444C6973743A4130312020204152502F23
:10109F0051202041322020553031203C20326E64C7
:1010AF003E3C63686F726420417270656767696F59
:1010BF003E3C7363616C6520417270656767696F51
:0E10CF003E3C737461626C2E5175616E7469E3
:1010DD007A653E3C636C6F636B205175616E74690C
:1010ED007A653E63686F72647363616C65207570B9
:1010FD0020646F776E616C7431616C743272616EE5
:10110D00646E6F202020646972656374207065724F
:10111D00204356202020207374657020627920733F
:10112D007465706F6666206F6E43484F5244202081
:10113D002020205343414C4520202020204B455951
:10114D004E4F54453A20204C4953543A41303120AA
:10115D0020534554555020202020204152504547C2
:10116D0047494F20205341564520202020202072F2
:10117D006F6F7420203173742020326E6420203301
:10118D007468205452414E53504F53453A202049D4
:10119D004E505554202020204F63746176652052A7
:1011AD00616E67654F6374617665205472616E730D
:1011BD00706F736520312D4F6374204469726563C0
:1011CD0074696F6E20322D4F6374204469726563AC
:1011DD0074696F6E20332D4F63742044697265639B
:1011ED0074696F6E20202053455454494E47534324
:1011FD00484F5244203E205530315343414C4520F9
:10120D003E205530312020204C495354203E204162
:10121D005072657373206B65792043484F5244219A
:10122D00202053544F52414745204F4B2021202021
:10123D002054554E452D4D4F444520204155544F7A
:10124D004C4F4144206C617374207361766564204A
:10125D004C6973742020202020202020204C69739D
:10126D00743A20415365742043562D4F5554733AAB
:10127D00202B38564B45594E4F54453A2020432389
:10128D00432044234420452046234620472347201E
:10129D004123412042030000000004000C000C0318
:1012AD00000C180C04000C182402000700070400A1
:1012BD00070E1502000500050400050A0F020004C3
:1012CD000004030004080C020003000303000306DE
:1012DD000C040003070E0400030A11040003060AA0
:1012ED000400030A0E040003070B030003060C049D
:1012FD000003070A0400030709030003070C03009A
:10130D0004070C0400040709040004070A04000480
:10131D00070B030005070C030002070C040004096A
:10132D000E030004080C030004060C040005070A54
:10133D00040004080A040004060A0400040B0E0449
:10134D0000040B0D0400040B0F040004070E040031
:10135D000B0E1104000B101504000B0E15040004E8
:10136D000B12030000000020202020202020202030
:10137D00554E49534F4E4F202020202020204F43C3
:10138D0054415645532031202020202020204F430A
:10139D0054415645532032202020202020204F43F9
:1013AD00544156455320332020202020202020203A
:1013BD00464946544820312020202020202020203E
:1013CD004649465448203220202020202020204607
:1013DD004F555254482031202020202020202046D7
:1013ED004F55525448203220202020205448495235
:1013FD0044206D616A20312020202020202041557D
:10140D00474D454E544544202020202054484952F4
:10141D0044206D696E203120202020202044494D2C
:10142D00494E495348454420202020204D494E4FD8
:10143D00522061646420392020202020204D494E07
:0E144D004F5220372F31312020202020204DFB
:10145B00494E4F522037206235202020202020205B
:10146B004D494E4F5220372F3920202020204D49F7
:10147B004E4F52206D616A203720202020202020E3
:10148B00204D494E4F522062352020202020202015
:10149B0020204D494E4F5220372020202020202045
:1014AB0020204D494E4F5220362020202020202036
:1014BB00202020204D494E4F52202020202020203C
:1014CB00202020204D414A4F522020202020202038
:1014DB0020204D414A4F5220362020202020202012
:1014EB0020204D414A4F52203720202020204D41B3
:1014FB004A4F52206D616A203720202020204D4119
:10150B004A4F5220737573203420202020204D41E8
:10151B004A4F522073757320322020202020202028
:10152B004D414A4F5220362F392020202020202099
:10153B00204D414A4F5220233520202020202020AF
:10154B00204D414A4F522062352020202020202060
:10155B004D414A4F5220372F342020202020204D40
:10156B00414A4F5220372023352020202020204D68
:10157B00414A4F5220372062352020202020202046
:10158B004D414A4F5220372F392020202020204D0B
:10159B00414A4F5220372062392020202020204DF5
:1015AB00414A4F52203720233920202020204D4103
:1015BB004A4F52206164642039202020204D414A3B
:1015CB004F5220372F392F31312020202020204D12
:1015DB00414A4F5220372F3133202020204D414A92
:1015EB004F5220372F392F313320202020204D41CF
:1015FB004A4F5220376220313120202020202020DA
:10160B002020554E49534F4E4F202020202020752F
:10161B007365722063686F72640800020305060726
:10162B00080B00000000060001040507080000007D
:10163B000000000500010307080000000000000087
:10164B000600030407090A0000000000000600035F
:10165B000506070A0000000000000700010405074B
:10166B00080B00000000000C000102030405060734
:10167B0008090A0B0500020407090000000000001E
:10168B0000070001040507080B000000000007001D
:10169B00010406080A0B0000000000050002050704
:1016AB000A00000000000000070002040507080AFA
:1016BB000000000000070003040607090A000000F1
:1016CB000000070002030607080B000000000005DE
:1016DB0000020307080000000000000005000105E0
:1016EB00060A0000000000000005000105070800C5
:1016FB0000000000000005000105070A00000000C3
:10170B0000000005000305070A00000000000000B0
:10171B0005000205070A000000000000000500029A
:10172B000407090000000000000007000204050682
:10173B00080A0000000000070001030406080A0065
:10174B0000000000070002040607080A0000000062
:10175B0000070002030507080B000000000007004C
:10176B0001030506090A000000000007000204053A
:10177B0008090B0000000000070002030607090A16
:10178B000000000000070001040507080A00000024
:10179B000000070003040607090B00000000000708
:1017AB000001030406080900000000000700020303
:1017BB000507090B000000000007000204050709DC
:0E17CB000B0000000000070002030507090ADA
:1017D9000000000000070001030507080A000000D7
:1017E9000000070002040607090B000000000007BB
:1017F9000002040507090A000000000007000203AF
:101809000507080A00000000000700010305060893
:101819000A0000000000070001030507090B00008A
:10182900000000070001030507080B000000000085
:101839000900020304060708090B0000000800015B
:1018490003040607090A0000000007000104050651
:10185900090A0000000000070002040607090A003F
:101869000000000005000103070800000000000057
:10187900000500020507090000000000000005003E
:101889000204070900000000000000050003050725
:101899000A0000000000000005000204060A00001A
:1018A9000000000000070001040507080A00000005
:1018B900000008000103040607090A0000000006E9
:1018C90000020406080A00000000000007000204E4
:1018D90006080A0B000000000020202020202020FC
:1018E90020416C67657269616E20202020202020CC
:1018F90020204172616269616E20202020202042EF
:10190900616C696E657369616E2020202020426CCC
:10191900756573206D616A6F722020202020426CEA
:10192900756573206D696E6F72202020202020203C
:1019390042797A616E74696E65202020202020200A
:101949004368726F6D617469632020202020202014
:1019590020446961746F6E696320446F75626C65B8
:10196900204861726D6F6E6963202020202020203D
:10197900456E69676D6174696320202020202020ED
:1019890020456779707469616E202020202020200D
:1019990048696E64757374616E2048756E6761720B
:1019A90069616E206D616A6F722048756E67617238
:1019B90069616E206D696E6F724A6170616E3A205D
:1019C90068697261796F7368694A6170616E3A69B1
:1019D9007761746F796F7368694A6170616E3A6B88
:1019E900756D6F69796F7368694A6170616E3A20C4
:1019F90020202020696E73656E4A6170616E3A20FD
:101A090020202020796F73656E4A6170616E3A20DB
:101A190020726974737573656E4A6170616E3A20DC
:101A290020202072796F73656E2020206D616A6FA6
:101A390072204C6F637269616E2020207375706526
:101A490072204C6F637269616E202020204C79648A
:101A590069616E206D696E6F724D696E6F72206873
:101A690061726D6F6E696320314D696E6F722068A6
:101A790061726D6F6E696320324D696E6F72206895
:101A890061726D6F6E696320334D696E6F72206884
:101A990061726D6F6E696320344D696E6F72206873
:101AA90061726D6F6E696320354D696E6F72206862
:101AB90061726D6F6E696320364D696E6F72206851
:101AC90061726D6F6E696320372020204D696E6FDA
:101AD90072206D656C6F6469634D6F64653A204966
:101AE9006F6E69616E2F4D616A4D6F64653A202092
:101AF900202020446F7269616E4D6F64653A202021
:101B090020506872796769616E4D6F64653A20206B
:101B19002020204C796469616E4D6F64653A204DCF
:101B290069786F6C796469616E4D6F64653A416576
:101B39006F6C69616E2F4D696E4D6F64653A202037
:0E1B490020204C6F637269616E4E6561706F93
:101B57006C6974616E206D616A6F724E6561706F3A
:101B67006C6974616E206D696E6F72202020202071
:101B770020204E696E6520546F6E6520202020203E
:101B870020204F637461746F6E69632020202020CA
:101B97002020204F7269656E74616C202020202000
:101BA7002020204F766572746F6E652020202020DC
:101BB70020202020202050656C6F672020202020C7
:101BC7002050656E7461746F6E69636D616A6F72C0
:101BD7002050656E7461746F6E69636D696E6F72A4
:101BE7002050656E7461746F6E6963202020202019
:101BF7002050726F6D6574686575732020202020F2
:101C0700202020205370616E6973682020202020D7
:101C170053796D6D6574726963616C202020202093
:101C2700202057686F6C65746F6E656C65616469B9
:101C37006E6757686F6C65746F6E65202020202073
:101C47002075736572207363616C65010000000085
:101C570001000000000000000000000000E53F3028
:101C6700E407121CA1121DD422121C77121C8C220D
:101C770020020122C205900117E004120D11F01293
:101C87001CE9C2022220030122C205900117E014B9
:101C9700120D11F0C203121CE922E53E30E10122C8
:101CA700E53E30E01530E31730E52DE53F30E7231B
:101CB70030E11130E21830E310227401021CE174A4
:101CC70002021CE17403021CE17404021CE17405A6
:101CD700021CE17406021CE17407900117F0121C44
:101CE700E922900117E01475F003A4901CF6730223
:101CF7001D0B021D1B021D2B021D3D021D56021D41
:101D070069021D767401900117F0121D8C12206371
:101D1700123816227402900117F0121D8C1224A596
:101D2700123832227403900117F0121D8CE54E12FF
:101D370034D012353C227404900117F0121D8C1216
:101D4700295A533C21533D41433C14433D282274B7
:101D570005900117F0121D8C533C21533D41433D23
:101D670028227406900117F0121D8C12283822744D
:101D770007900117F0121D8C533C21533D41433C02
:101D870002433D2822900117E0B401069011360264
:101D97001DC9B40206901140021DC9B40306901173
:101DA7004A021DC9B40406901154021DC9B40506A0
:101DB70090115E021DC9B40606901168021DC990F4
:101DC700117205A29000007B0A1204B1229001173C
:101DD700E01475F003A4901DE173021E0402221C97
:101DE7000233BA022889023A1E0228030238669093
:101DF7000FC005A29000097B041204B122121E171E
:101E0700121E2F121E471221531236311235D122BC
:101E170020020122C205900120E004120D96F090E5
:101E27000120F0C202D2342220030122C205900110
:101E370020E014120D96F0900120F0C203D2342254
:101E4700900120121E54900120121FA822E0B42BEB
:101E570006901614021F9450F81475F006A4901EED
:101E67006973901374021F62901384021F629013A8
:101E770094021F629013A4021F629013B4021F62A0
:101E87009013C4021F629013D4021F629013E402DE
:101E97001F629013F4021F62901404021F629014D1
:101EA70014021F62901424021F62901434021F62EE
:101EB700901444021F62901454021F62901464022B
:0E1EC7001F62901474021F62901484021F6246
:101ED500901494021F629014A4021F629014B4021D
:101EE5001F629014C4021F629014D4021F629014E2
:101EF500E4021F629014F4021F62901504021F622F
:101F0500901514021F62901524021F629015340269
:101F15001F62901544021F62901554021F629015AE
:101F250064021F62901574021F62901584021F627D
:101F3500901594021F629015A4021F629015B402B9
:101F45001F629015C4021F629015D4021F6290157E
:101F5500E4021F629015F4021F6290160405A29018
:101F650000107B101204B11221A790000D7450F0DF
:101F75002205A29000107B101204B1900FC005A29B
:101F850090000A7B031204B190000D7450F02205F5
:101F9500A29000107B101204B11221A790000D74BD
:101FA50055F022E0B42B03021FB850FB90000E122F
:101FB50006DD22C3942A90000E1206DD222034018C
:101FC50022C234121FE41221E11220631238169046
:101FD5000120E0F56990015A123BC3E569F02290B2
:101FE5000120E0B42B0302202D50FB1475F005A44D
:101FF500FB9012A293FC0BEB93254EFD0BEB932567
:102005004EFE0BEB93254EFF0BEB93254E90003CBC
:10201500F090003BEFF090003AEEF0900039EDF0D3
:10202500900038ECF0F56022123D9390027FE0FBC2
:10203500A3E0254EFCA3E0254EFDA3E0254EFEA31F
:10204500E0254E90003CF090003BEEF090003AED1C
:10205500F0900039ECF0900038EBF0F56022533C3D
:1020650021533D41E560B4000122B40108900039D7
:10207500E012210A22B4020F900039E012210A90E1
:10208500003AE012210A22B40316900039E0122129
:102095000A90003AE012210A90003BE012210A2240
:1020A500900039E012210A90003AE012210A9000CE
:1020B5003BE012210A90003CE012210A2290011710
:1020C500E0B40507300C04123B2D22900039E025C1
:1020D500532555120BF1120B3190003AE02553258B
:1020E50055120BF1120B3A90003BE0255325551282
:1020F5000BF1120B4390003CE025532555120BF1D3
:10210500120B4C2222F9E56375F00CA4C3C9991290
:102115000E5475F004A490211F73433C0222433CE6
:102125000422433C0822433C1022433C4022433CCA
:102135008022433D0222433D0422433D0822433D84
:102145001022433D2022433D8022433D0022900141
:1021550017E0B4010302215E22E53E30E10122E5EC
:102165003E30E20AE53F30E01FC210C211222010C6
:1021750016D210900142123BC3E004120D5DF0909F
:102185000124F01221D42222201116D211900142ED
:10219500123BC3E014120D5DF0900124F01221D41E
:1021A5002222900124E01475F006A49021B47390C6
:1021B500117C0221C99011810221C9901186022149
:1021C500C990118B05A29000087B051204B122125B
:1021D5001FE41221E112206312381622900124E037
:1021E500B4010122B40208900039E0240CF022B4B5
:1021F500030F900039E0240CF090003AE0240CF035
:1022050022900039E0240CF090003AE0240CF09084
:10221500003BE0240CF022122239122251122269CD
:10222500900FC005A29000087B051204B11236314B
:102235001235D12220020122C205900121E00412AB
:0E2245000DA9F0900121F0C202D23522200333
:102253000122C205900121E014120DA9F090012181
:10226300F0C203D23522900121122279121DF69079
:1022730001211223ED22E0B43707901C42121F9470
:102283002250F7B42B0302228E400BC3942B75F01C
:1022930006A490239E731475F006A49022A2739053
:1022A30018E20223E99018F20223E99019020223AB
:1022B300E99019120223E99019220223E9901932B5
:1022C3000223E99019420223E99019520223E9906B
:1022D30019620223E99019720223E99019820223F9
:1022E300E99019920223E99019A20223E99019B205
:1022F3000223E99019C20223E99019D20223E9903B
:1023030019E20223E99019F20223E9901A02022347
:10231300E9901A120223E9901A220223E9901A3251
:102323000223E9901A420223E9901A520223E99008
:102333001A620223E9901A720223E9901A82022395
:10234300E9901A920223E9901AA20223E9901AB2A1
:102353000223E9901AC20223E9901AD20223E990D8
:102363001AE20223E9901AF20223E9901B020223E4
:10237300E9901B120223E9901B220223E9901B32EE
:102383000223E9901B420223E9901B520223E990A6
:102393001B620223E9901B720223E9901B82022332
:1023A300E9901B920223E9901BA20223E9901BB23E
:1023B3000223E9901BC20223E9901BD20223E99076
:1023C3001BE20223E9901BF20223E9901C02022381
:1023D300E9901C120223E9901C220223E9901C328B
:1023E3000223E9901C42121F7622E0B43703022332
:1023F300FD50FB90000E1206DD22C3943690000EB2
:102403001206DD2220350122C2351224261224A50C
:10241300123832900121E0F5699001A2123BC3E525
:1024230069F022900121E0B4370A123DAD90003DDE
:10243300E0F5612250F412247705A290003DF0F5F7
:102443006112246622B4370A123DC790004AE0F5B0
:10245300622250F412247705A290004AF0F562122A
:10246300246622A305A20BEB9305A2254EF0A30538
:10247300A2DAF322B4130302247F50069016240237
:10248300249CB4260302248D500990171BC3941374
:1024930002249C901812C394261475F00DA4FB9388
:1024A300FA22533C21533D4190003DE0FA70012252
:1024B300A3E005A212210A05A2DAF522120A1212DA
:1024C30009B6B437030224D8500BD294533CFE53BD
:1024D3003DFEC20922433C0130090122D2091546BF
:1024E300E54660012212278D1225689001EA123B0E
:1024F300C3E0F546C294433D01E545B5470975453B
:102503000012330502250C50F5122534122515054A
:102513004522E025532549255612252022F990010D
:1025230017E0B40504300C0122E9120BF1120B552C
:1025330022E54CB4050412255122122541229000B4
:10254300B7E5822545F582E5833400F58322E54727
:10255300120C9DF5459000B7E5822545F582E5838C
:102563003400F58322900172123BC3E0B4010412DC
:10257300257D22B402031225A822E54CB40107905D
:1025830000B71225EE22B402079000B712261E22CE
:10259300B4030412268522B4040412269C2290005C
:1025A300B71225EE22E54CB401079000B71226CBF3
:1025B30022B402079000B71226FB22B403041227A9
:0E25C3006222B40404122779229000B7122677
:1025D100CB22E56070057E01790122FEF922E560DA
:1025E100B402057E0279022240F9FEF9221225D3B6
:1025F100AB4B0B7A0005A2900039122612EEF9EAD4
:10260100240CFA900039DBF2E54B048EF0A4F54777
:1026110022E02AA305A2F0A305A2D9F5221225D30F
:10262100AB4BEB75F00CA4FA0B05A2900038123BF2
:10263100F412264DEEF9EAC3940CFA900038123BDD
:10264100F4DBEEE54B048EF0A4F54722E02AFF12FD
:102651003BE605A2EFF0A305A2D9F1221225DF196D
:10266100AB4BEB75F00CA4FA0B05A2900038123BB2
:10267100F412264DEEF9EAC3940CFA900038123B9D
:10268100F4DBEE229000B71225EE05A212265DE5DD
:102691004775F002A4C39402F547229000B71225B2
:1026A100EE05A212261EE54775F002A4F54722E5C4
:1026B1006170057E01790122FEF922E561B402050E
:1026C1007E0279022240F9FEF9221226B0AB4B0BB1
:1026D1007A0005A290003E1226EFEEF9EA240CFAE8
:1026E10090003EDBF2E54B048EF0A4F54722E02A90
:1026F100A305A2F0A305A2D9F5221226B0AB4BEB9C
:1027010075F00CA4FA0B05A290003D123BF41227C0
:102711002AEEF9EAC3940CFA90003D123BF4DBEE89
:10272100E54B048EF0A4F54722E02AFF123BE605B3
:10273100A2EFF0A305A2D9F1221226BC19AB4BEBF3
:1027410075F00CA4FA0B05A290003D123BF4122780
:102751002AEEF9EAC3940CFA90003D123BF4DBEE49
:10276100229000B71226CB05A212273AE54775F051
:1027710002A4C39402F547229000B71226CB05A20A
:102781001226FBE54775F002A4F547221227F690C1
:102791000127E0B401149001D2123BC3E0F54CE5EE
:1027A1004A120E41F54B75490022B402189001D22C
:1027B100123BC3E0F54C754B00E54A120E2E75F045
:1027C1000CA4F54922B4030EE54A120DCFF54C7560
:1027D1004B0075490022B4040EE54A120DCFF54CA9
:1027E100754B0175490022E54A120DCFF54C754B29
:1027F1000275490022120A06120A4475F00C84F58A
:102801004A2212280A12282122200201229001279D
:10281100E004120E1BF0900127F0122838C20222A8
:1028210020030122900127E014120E1BF0900127D2
:10283100F0122838C20322533C21533D4190119A92
:1028410005A29000097B071204B112284F229001C2
:1028510027E0120E1BF01475F006A4902860739007
:1028610011A102287E9011B102287E9011C1022887
:102871007E9011D102287E9011E102287E05A2905E
:1028810000107B101204B122122921122896122E57
:10289100481235D122E53E30E1041228E222122805
:1028A100A322E53E30E222E53F30E005C210C2112D
:1028B10022201014D210900129E004120F1DF012F1
:1028C100402C12295A12326622201114D211900181
:1028D10029E014120F1DF012402C12295A123266EF
:1028E10022E53E30E222E53F30E005C210C211226E
:1028F100201014D21090011AE004120D83F0122B53
:102901003712295A12326622201114D21190011A5B
:10291100E014120D83F0122B3712295A123266225B
:10292100E53E20E10122E53F30E60AE53E30E417CD
:10293100C214C2152220140ED214900119E01412EF
:0E2941000D70F012295A2220150ED2159001A9
:10294F0019E004120D70F012295A22900119E0B407
:10295F000124122B4E900FF405A29000107B011250
:10296F0004B190012A122C9F900FF505A29000142C
:10297F007B011204B122B40221122B4E900FF405E9
:10298F00A29000157B011204B1122CD0900FF50507
:10299F00A290001A7B011204B122B40328122B4E0D
:1029AF00900FF405A290001B7B011204B190015A05
:1029BF00123BC3E0122D00900FF505A290001F7B74
:1029CF00011204B122B40404122B8222B40904129E
:1029DF002B9922B40A04122BD722900172123BC3F7
:1029EF00E0B40304122A942250FA1229FD22900116
:1029FF0019E0B40527122BEE900FF405A2900010EA
:102A0F007B011204B190018A122CBF900FF505A221
:102A1F009000147B011204B1122DD122B4062112A1
:102A2F002BEE900FF405A290001B7B011204B11244
:102A3F002DD1900FF505A290001F7B011204B1223A
:102A4F00B40721122C18900FF405A29000137B01EC
:102A5F001204B1122DF3900FF505A29000187B010F
:102A6F001204B122122C18900FF405A290001C7BB7
:102A7F00011204B1900FF505A290001F7B01120403
:102A8F00B1122E2922900119E0B40524122C3F9087
:102A9F000FF405A29000107B011204B190020212F4
:102AAF002CBF900FF505A29000147B011204B122E8
:102ABF00B40627122C3F900FF405A290001B7B0148
:102ACF001204B1900232123BC3122D26900FF5055E
:102ADF00A290001F7B011204B122B40724122C6FA5
:102AEF00900FF405A29000107B011204B190021A0E
:102AFF00122CBF900FF505A29000147B011204B1A8
:102B0F0022122C6F900FF405A290001B7B01120470
:102B1F00B190024A123BC3122D26900FF505A290D9
:102B2F00001F7B011204B12290011AE090000612DF
:102B3F0006DD22900129E0142441900005F02212B5
:102B4F002B42122B3790105605A29000097B0712CB
:102B5F0004B1900FF605A29000107B101204B190F3
:102B6F00012A122C9F122CD090015A123BC3E01253
:102B7F002D0022122B42122B3790105D05A29000D0
:102B8F00097B071204B1122D4C22122B42122B3744
:102B9F0090107205A29000097B071204B1900FC02C
:102BAF0005A29000107B0C1204B1900FF405A290B7
:102BBF00001C7B011204B1122D7C900FF505A29021
:102BCF00001F7B011204B122122B42122B379010DF
:102BDF007905A29000097B071204B1122D872212EA
:102BEF002B42122B3790106405A29000097B07121D
:102BFF0004B190100605A29000107B101204B19042
:102C0F00018A122CBF122DA822122B42122B3790A1
:102C1F00106405A29000097B071204B190101605ED
:102C2F00A29000107B101204B1122DF3122E292244
:102C3F00122B42122B3790106B05A29000097B07C5
:102C4F001204B190102605A29000107B101204B14F
:102C5F00900202122CBF900232123BC3122D262279
:102C6F00122B42122B3790106B05A29000097B0795
:102C7F001204B190103605A29000107B101204B10F
:102C8F0090021A122CBF90024A123BC3122D262219
:102C9F00123BC3E075F00C84FEE5F012359905A2E6
:102CAF009000117B021204B1EE9000131206D9228C
:0E2CBF00123BC3E09000121206DD900011746B
:102CCD002BF022900142123BC3E01475F006A49044
:102CDD002CE07390117C022CF5901181022CF59053
:102CED001186022CF590118B05A29000167B041213
:102CFD0004B122E0B42B03022D1650FB90001D12DF
:102D0D0006DD90001C7450F022C3942A90001D1211
:102D1D0006DD90001C7455F022E0B43703022D3C03
:102D2D0050FB90001D1206DD90001C7450F022C364
:102D3D00943690001D1206DD90001C7455F0229003
:102D4D000172123BC3E01475F006A4902D5C7390D4
:102D5D0010B0022D719010C0022D719010D0022D67
:102D6D00719010E005A29000107B101204B122901A
:102D7D00027AE090001D1206DD2290027BE01475B0
:102D8D00F006A4902D9473901110022D9D9011209A
:102D9D0005A29000107B101204B122900172123B1B
:102DAD00C3E0B4010E9010F005A29000167B051241
:102DBD0004B122B4020D9010F505A29000167B050A
:102DCD001204B122900172123BC3E0B4010A9001CA
:102DDD005A123BC3122D0022B4020A9001A2123BDB
:102DED00C3E0122D26229001D2123BC3E01475F0E0
:102DFD0006A4902E03739010FA022E1E9010FE0260
:102E0D002E1E901102022E1E901106022E1E9011E2
:102E1D000A05A29000147B041204B1229001EA125B
:102E2D003BC3E0B4010E90110E05A290001D7B0274
:102E3D001204B12290001D1206DD22900119E0B49A
:102E4D000107122EF2122F0E22B40207122F2A1290
:102E5D002F4322B40307122F5C122F7522B40407DF
:102E6D00122F8E122FA722B40907122FC0122FD3A3
:102E7D0022B40A07122FE6122FF922900172123B8B
:102E8D00C3E0B40304122EC62250FA122E9C2290D7
:102E9D000119E0B4050712300C12302822B40604D3
:102EAD0012304422B407071230C01230D922B408B0
:102EBD00071230F212310A2222900119E0B40507EF
:102ECD0012312212313E22B4060712315A123173D9
:102EDD0022B4070712318C1231A822B40806123120
:102EED00C41231DD222002012290012A123BC3E0DF
:102EFD0004120E8BF090012A122C9F123266C20220
:102F0D00222003012290012A123BC3E014120E8BE2
:102F1D00F090012A122C9F123266C2032220020168
:102F2D0022900142123BC3E004120D5DF0122CD031
:102F3D00123266C2022220030122900142123BC3CB
:102F4D00E014120D5DF0122CD0123266C203222055
:102F5D0002012290015A123BC3E004120D96F012A9
:102F6D002D00123266C202222003012290015A1254
:102F7D003BC3E014120D96F0122D00123266C203FF
:102F8D002220020122900172123BC3E004120DBCFB
:102F9D00F0122D4C123266C2022220030122900142
:102FAD0072123BC3E014120DBCF0122D4C1232669E
:102FBD00C203222002012290027AE004120E9BF03D
:102FCD00122D7CC202222003012290027AE01412FB
:102FDD000E9BF0122D7CC203222002012290027B57
:102FED00E004120EAEF0122D87C202222003012240
:102FFD0090027BE014120EAEF0122D87C203222038
:10300D0002012290018A123BC3E004120E8BF09054
:10301D00018A122CBF123266C202222003012290B5
:10302D00018A123BC3E014120E8BF090018A122C10
:0E303D00BF123266C20322900172123BC3E042
:10304B00B4010712305C1230752212308E1230A789
:10305B00222002012290015A123BC3E004120D966A
:10306B00F0122D00123266C20222200301229001BF
:10307B005A123BC3E014120D96F0122D0012326659
:10308B00C20322200201229001A2123BC3E00412D0
:10309B000DA9F0122D26123266C202222003012244
:1030AB009001A2123BC3E014120DA9F0122D2612AF
:1030BB003266C20322200201229001D2123BC3E0EE
:1030CB0004120DCFF0122DF3123266C2022220032E
:1030DB0001229001D2123BC3E014120DCFF0122D3E
:1030EB00F3123266C20322200201229001EA123B44
:1030FB00C3E004120DE2F0F546122E29C202222083
:10310B000301229001EA123BC3E014120DE2F0F529
:10311B0046122E29C2032220020122900202123BE8
:10312B00C3E004120E8BF0900202122CBF12326617
:10313B00C2022220030122900202123BC3E01412AE
:10314B000E8BF0900202122CBF123266C2032220A9
:10315B00020122900232123BC3E004120DA9F012BD
:10316B002D26123266C20222200301229002321255
:10317B003BC3E014120DA9F0122D26123266C203C6
:10318B00222002012290021A123BC3E004120E8B82
:10319B00F090021A122CBF123266C20222200301D7
:1031AB002290021A123BC3E014120E8BF090021AFB
:1031BB00122CBF123266C203222002012290024A55
:1031CB00123BC3E004120DA9F0122D26123266C277
:1031DB0002222003012290024A123BC3E014120D7B
:1031EB00A9F0122D26123266C2032290027BE0B4A4
:1031FB0001041232052212323A221209EE120A444B
:10320B00B55D0122533DBFF55D120ED490011AF04E
:10321B00123266900117E0B4010412206322B4024B
:10322B00041224A522B40406122B3712295A221297
:10323B0009EE1209B6B4370302324E5006533DBFA6
:10324B00C20D22433D40200D11D20D90011AE00416
:10325B00120EEF90011AF012321B22D20A90012AA1
:10326B00123BC3E075F00C8485F04E75F00CA4F5A1
:10327B005590015A123BC3E0900120F0900142128D
:10328B003BC3E0900124F0121FE41221E112381627
:10329B0090018A123BC3E0F556900202123BC3E049
:1032AB00F55790021A123BC3E0F558900172123B8E
:1032BB00C3E0900122F0123305B403041232E92269
:1032CB0050FA1232D1222033030232E89001A212BB
:1032DB003BC3E0900121F0122426123832229002D7
:1032EB0032123BC3E0900121F012242612383290A7
:1032FB00024A123BC3E012244822900122E0B4019F
:10330B0003C23322B40202D23322900122E0B4036F
:10331B000412335222B4040312332722120A12125C
:10332B0009B6B43703023340500BD294533CFE53CF
:10333B003DFEC20922C294433C01433D01300901C9
:10334B0022D20912335222120A06120A44120E8298
:10335B00B55A1012339822F55A85575990003D12E1
:10336B00337C2250F2F55A85585990004A12337C1F
:10337B002275F00C8485F06975F00CA4FAE0F9A3C2
:10338B00E0C3954EB56903023398D9F322B54D04CA
:10339B00200A0122C20AF54D254E2A255912252055
:1033AB00900122E0B40307C294433D01D23622E5DB
:0E33BB003E20E101221233D31234ADE54E1252
:1033C90034D012353CC202C20322E53E20E0057426
:1033D9000002343E20E205740102343E20E3057404
:1033E9000202343EE53F20E505740602343E20E042
:1033F90005740302343E20E105740402343E20E3DF
:1034090005740502343E20E205740702343E20E6C5
:1034190005740802343E20E705740902343EE53E8E
:1034290020E405740A02343E20E505740B02343E9B
:10343900E54EC22E22202E2ED22E854E4FF54E124B
:10344900347012347C900125E54EF0A3F0F9900117
:103459002A123BC3E075F00C8475F00CA4254EF0DC
:1034690012256812326622900038740412348712C9
:1034790038162290003DE012349A12383222FA703E
:103489000122A3E0FC254EC3954F120E64F0DAF237
:1034990022FA700122A3E0FC254EC3954F120E6457
:1034A900F0DAF2221209FA120A44B43C030234BCDB
:1034B900400122F553B5540122F55475F00C84F5F9
:1034C9005C85F05BD20A22533C21533D41120E54D4
:1034D90075F007A49034E173533D41433C022253F4
:1034E9003D41433C0422533D41433C0822533D4165
:1034F900433C1022533D41433C4022533D41433C10
:103509008022533C21433D0222533C21433D042266
:10351900533C21433D0822533C21433D1022533C57
:1035290021433D2022533C21433D8022533C2153DA
:103539003D4122900FC005A290000A7B041204B1FC
:10354900E54E12359905A290000E7B021204B19046
:10355900119005A29000107B0A1204B1900FC005CA
:10356900A290001A7B031204B1E55490001E1206C2
:10357900DD90001D742BF022E55B12359905A290B0
:10358900001D7B021204B1E55C90001F1206D922CE
:1035990075F004A49035A17390128A2290128C229E
:1035A90090128E22901290229012922290129422BE
:1035B900901296229012982290129A2290129C228E
:1035C90090129E229012A022900117E0B4010302EA
:1035D90035E8B402030235E8B404030235E822E50C
:1035E9003E30E10122E53E30E40AE53F30E616C20D
:1035F90012C2132220120DD212E56304120E72F5C3
:103609006312361F2220130DD213E56314120E72B2
:10361900F56312361F22900117E0B40104122063EA
:1036290022B402031224A522E53E20E1012212362A
:103639005C1236701236841236981236AC1236C0C5
:103649001236D41236E81236FC1237101237241209
:10365900373822E53E30E003C20F22200F08D20F8F
:1036690090005712374C22E53E30E203C216222061
:103679001608D21690005812374C22E53E30E30363
:10368900C21722201708D21790005912374C22E589
:103699003F30E003C21822201808D21890005A12AD
:1036A900374C22E53F30E103C21922201908D2190B
:1036B90090005B12374C22E53F30E303C21A222007
:1036C9001A08D21A90005C12374C22E53F30E50304
:1036D900C21B22201B08D21B90005D12374C22E529
:1036E9003F30E203C21C22201C08D21C90005E124B
:1036F900374C22E53F30E603C21D22201D08D21DAA
:1037090090005F12374C22E53F30E703C21E2220AA
:103719001E08D21E90006012374C22E53E30E403A9
:10372900C21F22201F08D21F90006112374C22E5C8
:0E3739003E30E503C22022202008D22090005E
:103747006212374C2205A2900117E0B4010905A2C5
:10375700123B8012376D22B4020B05A2123BA41252
:103767003B801237BC22E020E01DE560B4040F0562
:10377700A27B0490005612380B05A202378750EF40
:10378700E0D2E0F0023791C2E0F07C007B007A30B3
:1037970090005705A290003905A2E030E0080BEC35
:1037A70005A2F0A305A2A30CDAF0900038EBF0F520
:1037B7006012206322E020E01DE561B40C0F05A232
:1037C7007B0C90008612380B05A20237D650EFE02B
:1037D700D2E0F00237E0C2E0F07C007B007A309064
:1037E700008705A290003E05A2E030E0080BEC053B
:1037F700A2F0A305A2A30CDAF090003DEBF0F5616F
:103807001224A522A3E030E0FBDBF9C2E0F022128C
:10381700384E900038E0FBA3E004FA05A29000566A
:10382700A3DAFD7401F005A2DBED2212385A9000ED
:103837003DE0FBA3E004FA05A2900086A3DAFD743D
:1038470001F005A2DBED2290005774007930F0A358
:10385700D9FC2290008774007930F0A3D9FC22129A
:10386700387612394512399B1238B01239D722E50A
:103877003E20E10122E53F30E60AE53E30E414C28E
:1038870014C2152220140BD21490011CE014120F3D
:103897000AF02220150BD21590011CE004120F0A22
:1038A700F02290000E1206DD2290011CE0B4010107
:1038B70022B402071238D31238E622B403071238AB
:1038C700F912390C2212391F123932222002012231
:1038D70090011DE004120D4AF01238A9C2022220FD
:1038E70003012290011DE014120D4AF01238A9C2FB
:1038F70003222002012290011EE004120D4AF01259
:1039070038A9C202222003012290011EE014120DE1
:103917004AF01238A9C2032220020122900129E0AD
:1039270004120F1DF012398FC202222003012290C8
:103937000129E014120F1DF012398FC203229001E2
:103947001CE0B4010E9011F105A29000057B0B124B
:1039570004B122B4020E9011FC1239CC90011DE083
:103967001238A922B4030E9012071239CC90011E07
:10397700E01238A9229012121239CC12398F900016
:103987000E7420F012398F22900129E014244190FF
:10399700000FF022900035E060012290121D05A271
:1039A7009000107B101204B12290122D05A29000F6
:1039B700107B101204B122900FB005A29000107B6B
:1039C700101204B12205A29000057B091204B1224E
:1039D700E53E30E003C20B22200B1BD20B1239BE8F
:1039E7001201FDC2AF1239FED2AF1203601239B015
:1039F7009000357404F02290011CE0B40104123DDC
:103A07003022B40204123D5622B40304123D692247
:103A1700123FF8123D3022123A28123A5B123AAF9F
:103A270022E53E20E10122E53F30E60AE53E30E4AB
:103A370014C214C2152220140BD21490011FE014D3
:103A4700120EC1F02220150BD21590011FE00412AF
:103A57000EC1F02290011FE0B4011190123D05A2A2
:103A67009000067B0A1204B1123AE422901247052D
:103A7700A29000067B0A1204B1123A842290012810
:103A8700E0B4010E90125105A29000107B101204B1
:103A9700B1221414244190001FF090126105A290E6
:103AA70000107B0F1204B12290011FE0B40107122E
:0E3AB7003AC4123AD422123B60123B70222015
:103AC500020122900118E004120D24F0C202222006
:103AD500030122900118E014120D24F0C203229074
:103AE500127105A29000107B0D1204B1900118E02F
:103AF500B4011090113005A290001D7B031204B192
:103B0500C20C22141490001E1206D990127E05A232
:103B150090001D7B011204B190128005A290001F38
:103B25007B011204B1D20C22900118E0141475F037
:103B35000CA4F565120BF1120B31E565120BF112B0
:103B45000B3AE565120BF1120B43E565120BF11209
:103B55000B4CE565120BF1120B5522200201229048
:103B65000128E004120D37F0C20222200301229041
:103B75000128E014120D37F0C20322E56375F00C3D
:103B8500A48582328583337534007535007832F526
:103B95003675370079361202238682088683228598
:103BA5008232858333753400753500783275363049
:103BB500753700793612022386820886832285822C
:103BC50032858333753400753500783290011AE0FB
:103BD50014F53675370079361202238682088683F6
:103BE50022C3E5829401F582E5839400F58322E5FD
:103BF5008229F582E5833400F58322858232858327
:103C050033753400753500783290011DE01475F078
:103C150005A4023C318582328583337534007535C0
:103C250000783290011EE01475F00DA4F536753755
:103C350000793612022386820886832285823285A0
:103C45008333753400753500783275F005023C66AE
:103C5500858232858333753400753500783275F089
:103C65000DA4F5367537007936120223868208864B
:103C750083227532557533017534007535007832F8
:103C850014F536753700793612023E86820886832A
:103C950022901C5205A29000007E1005A27F0512FD
:103CA5003CC6901C5205A2DEF22290003D05A29072
:103CB50000A07E1005A2790D123CFD90003DDEF6B8
:103CC5002274009343D20205A2F0A375D25275D295
:103CD500A2E5D220E0FB53D2FD05A2A3DFE32290AB
:103CE500003D05A2901C577B0DE493A305A2F0A30C
:103CF50005A2DBF5123CAF22E0A343D20205A2F0F8
:103D0500A375D25275D2A2E5D220E0FB53D2FD05B0
:103D1500A2D9E52243D202438E20E0A353D2FD531C
:103D25008EDF05A2F0A305A2D9EA22790A90012027
:103D350005A290024005A2123CFD22900125E54E08
:103D4500F0A3E54FF022900125E0F54EA3E0F54FF5
:103D55002290003805A2900000123C0005A27905CA
:103D6500123CFD2290003D05A29000A0123C1A05D0
:103D7500A2790D123CFD22C2AF790A90024005A23C
:103D850090012005A2123D19123D4BD2AF22C2AFC0
:103D9500900000C3942B123C4105A290027F05A21E
:103DA5007905123D19D2AF22C2AF9000A0C3943756
:103DB500123C5505A290003D05A2790D123D19D280
:103DC500AF22C2AF9000A0C39437123C5505A29014
:103DD500004A05A2790D123D19D2AF22E53E30E128
:103DE5000122753C10900F9005A29000007B1012E7
:103DF50004B1900FA005A29000107B101204B1E54C
:103E05003E30E1FBE53F30E00630E632023E09E5B3
:103E15003F30E0FB1201FD1201FD900FB005A290AD
:103E250000107B101204B11201FD1201FDC2AF1288
:0E3E35003C96123CE4123E4F123E8FD2AF225A
:103E4300E53F30E6FB1201FD1201FD2290012074D3
:103E530016F09001217401F09001227401F0900199
:103E6300237401F09001247401F09001257400F093
:103E73009001267400F09001277401F090012874DA
:103E830001F09001297401F0123D302290027A74FE
:103E930018F090027B7401F090012A7400123F2302
:103EA30090018A7400123F239002027400123F2390
:103EB30090021A7400123F239001427401123F23AF
:103EC30090015A741B123F239001727401123F2315
:103ED3009001A2742F123F239001BA741B123F2347
:103EE3009001D27403123F239001EA7401123F231D
:103EF3009002327401123F2390024A7401123F234D
:103F0300123F07227401900129F0123C77124003FB
:103F1300900129E004F0B40DF17401900129F0221D
:103F23007B18F0A3DBFC22123FCA74A0F9123F975F
:103F3300123FE0E566F9123F97123FE0E567F91299
:103F43003F97123FE0123FCA74A1F9123F97123F05
:103F5300E0123F8A123FE6123FBC22E9FA123FCA3F
:103F630074A0F9123F97123FE6E566F9123F9712E4
:103F73003FE6E567F9123F97123FE6EAF9123F97EA
:103F8300123FE6123FBC22D2A57808123FECE93378
:103F9300F9D8F8227808E93392A5F9123FECD8F65C
:103FA300227B80DB02800E123FCA74A0F9123F9776
:103FB300123FE640EE123FBC22C2A500D2A400008D
:103FC30000000000D2A522D2A500D2A40000000068
:103FD3000000C2A5000000000000C2A422C2A51276
:103FE3003FEC22D2A5123FEC220000D2A400000035
:103FF300A2A5C2A422900129E0123C771240032219
:1040030005A290012A05A27FD81240157F7D124098
:10401300152285836685826705A2E0F9A305A212AE
:104023003F5E123FA4A3DFEA22900129E0123C770E
:1040330012405122900128E0B40107900129E002C7
:10404300404A14900129F0123C771240512205A2F4
:1040530090012A05A27FD81240637F7D124063221C
:10406300858366858267123F2AA3E905A2F0A3052B
:10407300A2DFED2275402875410475427D75430228
:1040830075440A90FF9C8582CA8583CB8582CC8543
:1040930083CD43C804D2ADD2AF22C0E0C0D0E58205
:1040A300C0E0E583C0E0D2D4C2D3C2CFD5404675C9
:1040B3004028120306120900120911B20E12094F09
:1040C30030360DD5440A754405D294533DFEC236AD
:1040D300D54122754106120988120C39120C6ED58E
:1040E3004213754232900035E0600214F0D5430567
:1040F300754314B205D0E0F583D0E0F582D0D0D07B
:02410300E032A8
:00000001FF
